:0C00000022C0FECF5BC0FCCFFBCF3AC09B
:10000C00F9CFF8CFF7CFF6CFF5CFF4CFF3CFF2CFC0
:10001C00F1CFF0CFEFCFEECFEDCFECCFEBCF102772
:10002C00E80364000A000100001000011000010048
:10003C007266496E69740D0A0000F894EE27ECBBE9
:10004C00E5BFF8E1A895A4B7A77FA4BFF1BDE1BDBA
:10005C008DE0A2E0ED938A95E9F780E8A0E6ED93B8
:10006C008A95E9F7E0E0E3BBE4BBE5BBEFEDEDBF60
:10007C00C0E875C1AA93EA93EFB7EA93EFE1EDBD3F
:10008C00E0E0ECBDA0E09899A1E0E1E0EA2711F4F2
:10009C00989801C0989A849B06C03394E2E0E315CB
:1000AC0011F494983324E991EFBFE991A991189533
:1000BC000A921A92FA926A937A938A939A93AA93CF
:1000CC00BA93EA93FA93EFB7EA93E0E0EBBF839924
:1000DC0002C0859901C002C0A1E080D1839902C001
:1000EC00859B01C002C0A2E079D1E0E8EBBFE991A9
:1000FC00EFBFF991E991B991A99199918991799170
:10010C006991F990199009901895BA93AA931A933A
:10011C0010E0EB811E1750F4969AA981BA81D5D1C3
:10012C009698A981BA81D1D11F5FF3CF188156C09F
:10013C00BA93AA93DFD100E010E0C498EB81F07081
:10014C00EFB9E1E1EDB9E3E1EDB9E1E1EDB9E3E1FD
:10015C00EDB9E1E1EDB9E3E1EDB9E1E1EDB9E3E1EF
:10016C00EDB9E1E1EDB9E3E1EDB9E1E1EDB9E3E1DF
:10017C00EDB9E1E1EDB9E3E1EDB9E1E1EDB9E3E1CF
:10018C00EDB9EFB1FE2FE0E08F01EA81EFB9E1E1CB
:10019C00EDB9E3E1EDB9E1E1EDB9E3E1EDB9E1E1AF
:1001AC00EDB9E3E1EDB9E1E1EDB9E3E1EDB9E1E19F
:1001BC00EDB9E3E1EDB9E1E1EDB9E3E1EDB9E1E18F
:1001CC00EDB9E3E1EDB9E1E1EDB9E3E1EDB9EFB1A1
:1001DC00F0E00E2B1F2BC49AF8018FD124960895B2
:1001EC00AA938299FECFE881EFB9E1E1EDB9E3E1A1
:1001FC00EDB9E1E1EDB9E3E1EDB9E1E1EDB9E3E14F
:10020C00EDB9E1E1EDB9E3E1EDB9E1E1EDB9E3E13E
:10021C00EDB9E1E1EDB9E3E1EDB9E1E1EDB9E3E12E
:10022C00EDB9E1E1EDB9E3E1EDB938C1A0E0BEEF24
:10023C007FDFA6E9B0E049D1A8EDB0E879DFA9ED00
:10024C00B2E876DFA0E2B6EA73DFA5E0B6EC70DFC9
:10025C00A0EAB4E96DDFACEEB2EC6ADFA3E8BAEC6D
:10026C0067DFA6EDBEEC64DFABE9B4EC61DFA0E5C3
:10027C00B8E95EDFA7E7BCEC5BDFA0E0B0EE58DFCF
:10028C00A0E0B8EC55DFA0E0B0EC2FC0C698B39B53
:10029C0002C0B19901C0FBCFC298C498E1E1EDB99D
:1002AC00E3E1EDB9E1E1EDB9E3E1EDB9E1E1EDB99E
:1002BC00E3E1EDB9E1E1EDB9E3E1EDB9E1E1EDB98E
:1002CC00E3E1EDB9E1E1EDB9E3E1EDB9E1E1EDB97E
:1002DC00E3E1EDB9E1E1EDB9E3E1EDB9EFB1089599
:1002EC00A1E8BAEC25DFA3E8BAEC22DF0895E0E838
:1002FC00E6BDE0E0E6BDE4E0EBBBE0E0EABBE4E158
:10030C00E8BBE4EDE7BBE2E5E1BBEDE2E2BBE0E03C
:10031C00E0BFE3BFE2BFE6BFECBFEFBDE4E0EEBD84
:10032C00EFE1EDBDE0E0ECBDE5BDE4BDEBBDEABD4C
:10033C00E9BDE8BDE0E8E9BFE0E0E5BFE0E8EBBF20
:10034C00EABFE0E0EDB9EBB9E8E1EAB9E6E0E3B920
:10035C00E0E0E2B9E0E8E8B9E0E0E1B90895F8944A
:10036C00C6DFE7E0E9B962DFACE3B0E099D0E3E0E7
:10037C00EA93A4E6B0E0C9DE7894B2DF87DF1E2FE3
:10038C00A12F87D0A0E0B0E0AAD0E11711F57EDF55
:10039C000E2F7CDF3E2F7ADF2E2F78DF5E2FC29A56
:1003AC00C49A9EDFA1E0B0E09AD0E01779F4A2E005
:1003BC00B0E095D0E31751F4A3E0B0E090D0E21791
:1003CC0029F4A4E0B0E08BD0E51709F001C0949AB1
:1003DC00D5CFC29AC49A84DFD1CFFFCFFF92AA9314
:1003EC00869907C06894F0F8969AC29AA9E3B2E885
:1003FC009FDEC29AA0E0B0E09BDEC498A8EBF0DED2
:10040C00AAEAEEDEADE2ECDEA6EDEADEA0E0B0E0BC
:10041C0066D0AE2FE5DEA881A130A1F4A1E0B0E05A
:10042C005ED0AE2FDDDEA2E0B0E059D0AE2FD8DE2C
:10043C00A3E0B0E054D0AE2FD3DEA4E0B0E04FD0B8
:10044C00AE2FCEDEA881A230A1F4A5E0B0E047D05B
:10045C00AE2FC6DEA6E0B0E042D0AE2FC1DEA7E0E4
:10046C00B0E03DD0AE2FBCDEA8E0B0E038D0AE2F6F
:10047C00B7DEA0E0B5DEC298C49AA9E1B0E025D001
:10048C00F0FE04C0A9EDB2E853DE96982196FF90D9
:10049C000895AA935D9BFECFE881ECB9219608954F
:1004AC00BA93AA931A93E981FA813196E983FA8374
:1004BC003197E4911E2FE03019F0A12FEADFF3CF32
:1004CC00AAE0E7DF188123960895109639F086E6A6
:1004DC009EE00197F1F7A8951197C9F70895E19956
:1004EC00FECFFF93FFB7F894AEBBE09AEDB3FFBF1E
:1004FC00FF9108951A930A9308951981088108951C
:00000001FF
